:020000040000FA
:10000000830100308A00C028FF0003088301E2005A
:100010000408E3000A08E4008A015608EF005708C4
:10002000F0005808F1005908F2005A08F3005B0884
:10003000F4005C08F6005D08EE005E08ED005F0865
:10004000EC006008EB006108EA007508E900670849
:10005000E5006808E6000B1C2E282F2832288A119C
:10006000D3228A11831203130C1C372838289728AF
:1000700078308F00FF308E00861A43283F28061AFA
:1000800043284228452844286D283D302702031C78
:100090004A284B286928A701A0184F28502868280B
:1000A000A0140130A006201C562857285A280A30D0
:1000B000A6005D2883120313A601831203132608EA
:1000C000D40005308A1141218A118A1106218A1132
:1000D0006C2883120313A70A942883120313A01019
:1000E000A701861A74287728061A782877287A288C
:1000F00079289128A90A15302902031C8028812813
:100100009028A90306302802031C872888288D28F8
:10011000A8018A11D3228A11902883120313A80AF6
:10012000942883120313A901831203130C100313E1
:1001300083126F08D6007008D7007108D8007208C3
:10014000D9007308DA007408DB007608DC006E085A
:10015000DD006D08DE006C08DF006B08E0006A0857
:10016000E1006908F5006508E7006608E800630833
:10017000840064088A0062088300FF0E7F0E090075
:10018000203084002130CE20213084005630CE2013
:1001900083018A11072C04068001840A04060319CE
:1001A0000034CB288312E700E81BDF28681BE72810
:1001B00068088A006708E70A0319E80A82008313BF
:1001C000681883176708E70A840000080800820798
:1001D0003F3406345B344F3466346D347D34073439
:1001E0007F346F3477347C3439345E34793471340D
:1001F0008034313400340034FF3FFF3FFF3FFF3F86
:10020000FF3FFF3FFF3FFF3FFF3FFF3F83120313CF
:1002100007108A112A218A118A112A218A110714AA
:1002200003138312080083120313DA01DB010310A6
:10023000D90CD80C031C23295608DA0757080318D1
:10024000570ADB070310D60DD70D580859040319B8
:1002500000341729E83083120313D2000330D3008F
:1002600032293229FF3083120313D207031CD30330
:1002700053085204031D3D293E29312903138312DB
:10028000080083120313D500831603178C18462920
:1002900083120313550803178D0003135408031723
:1002A0008C0083168C1303108B1B03148B130C15FB
:1002B00055308D00AA308D008C140C1103188B174B
:1002C00083010800831203133908A2002208D40016
:1002D00002308A1141218A113808A5002508D4006E
:1002E00003308A1141218A1100303B02031D82290B
:1002F00000303A02031D822900303902031D822991
:10030000013038020318852986298A2995010C3085
:100310009700F5290030831203133B02031D9A292D
:1003200000303A02031D9A2900303902031D9A2930
:100330000230380203189D299E29A1293C309700DC
:10034000F529033083120313DA000030DB0000309C
:10035000DC000030DD003808D6003908D7003A0844
:10036000D8003B08D9008A11C1278A115608BC0061
:100370005708BD005808BE005908BF003C08D60009
:100380003D08D7003E08D8003F08D90002308A1542
:10039000F3278A11560895003C080339AB00E5297C
:1003A0000C30831203139700F5291C3083120313BA
:1003B0009700F5292C30831203139700F5293C3060
:1003C000831203139700F529F529831203132B08D1
:1003D000003A0319D029013A0319D529033A031920
:1003E000DA29013A0319DF29F529031383120800DA
:1003F000643083120313DA000030DB000030DC00CD
:100400000030DD004408D6004508D7004608D80073
:100410004708D9008A1146278A115608AA000030D9
:100420008A002A08E7208A11CD006430DA00003003
:10043000DB000030DC000030DD004408D600450859
:10044000D7004608D8004708D9008A1146278A11E4
:100450005A08AA000A30D7002A088A11BB268A1136
:10046000D60000308A005608E7208A118038CC0078
:100470000A30D7002A088A11BB268A115608D600EE
:1004800000308A005608E7208A11CB00003047026E
:10049000031D542A00304602031D542A0030450231
:1004A000031D542A013044020318572A582A5E2A91
:1004B0003F30CD00BF30CC003F30CB0064308312E2
:1004C0000313DA000030DB000030DC000030DD0018
:1004D0002C08D6002D08D7002E08D8002F08D900E8
:1004E0008A1146278A115608AA0000308A002A0875
:1004F000E7208A118038CA006430DA000030DB005F
:100500000030DC000030DD002C08D6002D08D700BC
:100510002E08D8002F08D9008A1146278A115A08B8
:10052000AA000A30D7002A088A11BB268A11D600F1
:1005300000308A005608E7208A11C9000A30D70027
:100540002A088A11BB268A115608D60000308A0074
:100550005608E7208A11C8008512D10106305102E1
:10056000031CB32AB42AB52ACD2A831203135108D7
:10057000483E8400831300089300831203138C1DEC
:10058000C22AC32ABD2A831203138C11D10A063052
:100590005102031CCC2ACD2AB52A831203138516D7
:1005A0000313831208008A112A218A112018D92ADC
:1005B000DA2AFF2B861AE12ADD2A061AE12AE02A26
:1005C000E32AE22AE42AFF2B83120313861AE92A7C
:1005D000EC2A061AED2AEC2AEF2AEE2AFF2B0B1042
:1005E0008A1106218A11FE308600861AF82AF92A15
:1005F000FB2A0230A40083120313061A002B012BDE
:10060000032BA401A40AFD30831203138600861A6B
:100610000A2B0B2B0D2B0430A40083120313061A94
:10062000122B132B152B0330A400FB308312031362
:100630008600861A1C2B1D2B1F2B0630A40083124C
:100640000313061A242B252B272B0530A400831215
:1006500003138601E52B0030831203133B02031DB5
:100660003B2B00303A02031D3B2B01303902031DA6
:100670003B2B3C30380203183E2B3F2B4B2B0A30D0
:10068000B80701300318B9070318BA070318BB07E6
:100690008A1162218A11FB2B0030831203133B0263
:1006A000031D5C2B00303A02031D5C2B0030390225
:1006B000031D5C2B0A303802031C5F2B602B772B49
:1006C000F630B807FF3003110318013E031DB907C8
:1006D000FF3003110318013E031DBA07FF30031159
:1006E0000318013E031DBB078A1162218A11FB2BEF
:1006F0000030831203133B02031D882B00303A02A3
:10070000031D882B01303902031D882B4630380227
:1007100003188B2B8C2B962BB80A0319B90A0319D3
:10072000BA0A0319BB0A8A1162218A11FB2B003015
:10073000831203133B02031DA72B00303A02031D53
:10074000A72B00303902031DA72B01303802031CF0
:10075000AA2BAB2BC22BFF30B807FF3003110318B5
:10076000013E031DB907FF3003110318013E031DAD
:10077000BA07FF3003110318013E031DBB078A119E
:1007800062218A11FB2B20308312031321020318EC
:10079000CA2BCB2BD22BA10A2108D4000C308A11F2
:1007A00041218A11FB2B0130831203132102031C08
:1007B000DA2BDB2BE22BA1032108D4000C308A11A9
:1007C00041218A11FB2BFB2BFB2B831203132408E3
:1007D000013A03192B2B033A03194C2B013A031945
:1007E000782B073A0319972B013A0319C32B033AC5
:1007F0000319D32BE32B0A3083120313A4008312B3
:100800000313060886000B100313831208008316D7
:1008100003130C140B17783083128F00FF308E00F7
:1008200025309000C0308316870001308312870086
:10083000113083169900B0309800803083129800F0
:10084000F030831686007F308100831286018B157D
:100850000B10060886008C0130309400C0308316DF
:1008600094000330850082309F00831295010C3084
:100870009700FF30831692000430831292007F307D
:100880009B000C309D00831603178C138B170C30C4
:100890008A15E7278A11A200343022020318512C4E
:1008A000522C542C2208A10002308A15E7278A1105
:1008B000A200CF01D00100305002643003194F0272
:1008C000031C632C642C652C742C0000831203130E
:1008D000CF0A0319D00A00305002643003194F02C6
:1008E000031C732C742C652C03308A15E7278A119E
:1008F000A5002508B800B901BA01BB012203031DF8
:10090000822C832C882CB90A0319BA0A0319BB0A52
:10091000033083120313DA000030DB000030DC0008
:100920000030DD003808D6003908D7003A08D80072
:100930003B08D9008A11C1278A115608BC00570804
:10094000BD005808BE005908BF003C08D6003D084D
:10095000D7003E08D8003F08D90002308A15F32797
:100960008A115608950005308A15E7278A11A200DA
:1009700022080A3A031DBD2CBE2CBF2C2014B82E11
:10098000C130831203139F00CF01D00117305002F2
:10099000703003194F02031CCE2CCF2CD02CDF2C2F
:1009A000000083120313CF0A0319D00A1730500234
:1009B000703003194F02031CDE2CDF2CD02C831265
:1009C00003130C131F15CE011E304E02031CE92C1D
:1009D000EA2CEB2CF52C000083120313CE0A1E30F8
:1009E0004E02031CF42CF52CEB2C03308312031362
:1009F000D8000030D9001E08E800E70183161E0861
:100A00008312D600D7016708D6070318D70A6808EB
:100A1000D7078A11F3268A115A08D6005B08D70037
:100A20000030D71BFF30D800D9005608B000570857
:100A3000B1005808B2005908B3000C130330DA00B3
:100A40000030DB000030DC000030DD003808D6006C
:100A50003908D7003A08D8003B08D9008A11C127C5
:100A60008A115608BC005708BD005808BE00590836
:100A7000BF003C08D6003D08D7003E08D8003F081C
:100A8000D90002308A15F3278A11560895003C08D0
:100A90000339AB00602D0C30831203139700702DC7
:100AA0001C30831203139700702D2C308312031314
:100AB0009700702D3C30831203139700702D702D1A
:100AC000831203132B08003A03194B2D013A031923
:100AD000502D033A0319552D013A03195A2D702D43
:100AE0000330831203132302031C772D782DF02D7E
:100AF0000330DA000030DB000030DC000030DD00C5
:100B00004008D6004108D7004208D8004308D90061
:100B10008A1146278A115608C4005708C50058088C
:100B2000C6005908C700C001C101C201C301A30129
:100B300000304702031DA62D00304602031DA62DDE
:100B400000304502031DA62D023044020318A92DD2
:100B5000AA2DB32D4408C4004508C5004608C600A8
:100B60004708C700EC2D0030831203134702031D12
:100B7000C32D00304602031DC32D00304502031D66
:100B8000C32D283044020318C62DC72DD12D0230A5
:100B9000C40701300318C5070318C6070318C707A1
:100BA000EC2D0030831203134702031DE12D0030AA
:100BB0004602031DE12D01304502031DE12D0E30DB
:100BC00044020318E42DE52DEC2DC40A0319C50ACF
:100BD0000319C60A0319C70A8A11F8218A11012EBE
:100BE00083120313A30A3008C00731080318310F1A
:100BF000C10732080318320FC20733080318330A3B
:100C0000C307C930831203139F00CF01D0011730EF
:100C10005002703003194F02031C0F2E102E112E9C
:100C2000202E000083120313CF0A0319D00A1730B5
:100C30005002703003194F02031C1F2E202E112E5C
:100C4000831203130C131F15CE011E304E02031C1A
:100C50002A2E2B2E2C2E362E000083120313CE0AA2
:100C60001E304E02031C352E362E2C2E83120313FB
:100C70001E08D900D80183161E088312D600D7019A
:100C80005808D6070318D70A5908D7075608D600B8
:100C90005708D7000030D71BFF30D800D9005608BE
:100CA000B4005708B5005808B6005908B7000C132F
:100CB0003A30DA000030DB000030DC000030DD00CC
:100CC0003408D6003508D7003608D8003708D900D0
:100CD0008A11C1278A116430DA000030DB0000304D
:100CE000DC000030DD008A1146278A115608AC006E
:100CF0005708AD005808AE005908AF0000302F0269
:100D0000031D8C2E00302E02031D8C2E00302D0270
:100D1000031D8C2E04302C0203188F2E902E942E3F
:100D2000AC01AD01AE01AF013B3083120313D8001B
:100D30000130D9002108D600D7018A1113218A1168
:100D40005A08D6005B08D7000A30D8000030D90016
:100D50008A11F3268A115A08D6005B08D70004309E
:100D6000D8000030D9008A11F3268A115A089B0056
:100D7000C02C8A11C02883120313D600DA01031095
:100D8000FD305707031CE42ED901F0305705031D31
:100D9000CC2E0430D900D70ED8010310D90AD70DB4
:100DA000031CCE2ED70C570856020318D600D80DB8
:100DB000D90BD22EDA1FDE2ED809D80A5808DA1F2E
:100DC0000800D609D60A0800D70C0318ED2ED70C58
:100DD000031CD6010310D60C031C03105608D800C0
:100DE000D601D60DDA2E83120313DC01D71FFF2E96
:100DF000D609D60A0319D703D7095C17DC17590897
:100E00008039DC06D91F0D2FD809D80A0319D90358
:100E1000D9090D2F83120313DC01DA01DB01580815
:100E20005904031D162FD601D70100341F30DC04EE
:100E30000310DC0AD80DD90D031C192FD90CD80CBE
:100E400059085702031D262F58085602031C2E2F3F
:100E50005808D6025908031C590AD702DA0DDB0DCF
:100E6000DC0BDC1A1E2FDC1F3A2FDA09DA0A031911
:100E7000DB03DB095A08D8005B08D9005C1F00348B
:100E8000D609D60A0319D703D7090034840183127F
:100E9000F501DE01DF01E001E1015A085B045C04B9
:100EA0005D040319562FC030F505612FD601D70117
:100EB000D801D901F12F0310DA0DDB0DDC0DDD0DAA
:100EC000F50ADD1F5B2FF50A0310DE0DDF0DE00DC7
:100ED000E10D5D085902031D772F5C085802031DC0
:100EE000772F5B085702031D772F5A085602031C01
:100EF000892F5E145A08D6025B08031C5B0FD702C9
:100F00005C08031C5C0FD8025D08031C5D0FD9024E
:100F10000310DD0CDC0CDB0CDA0CF50375083F3933
:100F2000031D642F751FA12F0310FF30D607D609AC
:100F3000031CD707D709031CD807D809031CD907F6
:100F4000D9095608DA005708DB005808DC005908B0
:100F5000DD005E08D6005F08D7006008D800610891
:100F6000D900F51FF12F0310FF30D607D609031C57
:100F7000D707D709031CD807D809031CD907D909F3
:100F8000F12F8401831203135608DE005708DF0097
:100F90005808E0005908E100D801D901D601D7016D
:100FA0000310E10CE00CDF0CDE0C031CE52F5A08EB
:100FB000D6075B0803185B0FD7075C0803185C0FA4
:100FC000D8075D0803185D0FD9075E085F04600449
:100FD00061040319F12F0310DA0DDB0DDC0DDD0DBB
:100FE000D02F84080319003459088000840358085E
:100FF0008000840357088000840356088000003472
:10100000FF3FFF3FFF3FFF3FFF3FFF3FFF3FFF3FF0
:10101000FF3FFF3FFF3FFF3FFF3FFF3FFF3FFF3FE0
:10102000FF3FFF3FFF3FFF3FFF3FFF3FFF3FFF3FD0
:10103000FF3FFF3FFF3FFF3FFF3FFF3FFF3FFF3FC0
:101FC000FF3FFF3FFF3FFF3FFF3FFF3FFF3F8312CA
:101FD0000313D10003178D0083168C130C14831286
:101FE0000C080313080083120313DA00DA0ADA0379
:101FF000031900340310D90CD80CD70CD60CF72FCA
:10420000FF00FF0000003300FF00FF00FF00FF0081
:10421000FF00FF00FF00FF002000FF00FF00FF0085
:10422000FF00FF00FF00FF00FF00FF00FF00FF0096
:10423000FF00FF00FF00FF00FF00FF00FF00FF0086
:10424000FF00FF00FF00FF00FF00FF00FF00FF0076
:10425000FF00FF00FF00FF00FF00FF00FF00FF0066
:10426000FF00FF00FF00FF00FF00FF00FF00FF0056
:10427000FF00FF00FF00FF00FF00FF00FF00FF0046
:10428000FF00FF00FF00FF00FF00FF00FF00FF0036
:10429000FF00FF00FF00FF00FF00FF00FF00FF0026
:1042A000FF00FF00FF00FF00FF00FF00FF00FF0016
:1042B000FF00FF00FF00FF00FF00FF00FF00FF0006
:1042C000FF00FF00FF00FF00FF00FF00FF00FF00F6
:1042D000FF00FF00FF00FF00FF00FF00FF00FF00E6
:1042E000FF00FF00FF00FF00FF00FF00FF00FF00D6
:1042F000FF00FF00FF00FF00FF00FF00FF00FF00C6
:02400E003A3F37
:08400000FF3FFF3FFF3FFF3FC0
:00000001FF
